:02000000040AF0
:080008009F0C0200080C060029
:10001000000C260066060A0A3E0966060A0A6607FA
:100020000F0A3E093E093E093E093E093E093E09C6
:100030003E0966070F0A3E093E093E093E0966076A
:10004000320A3E093E093E096607350A3E093E0965
:100050003E096607380A3E093E093E093E09660721
:100060003B0A0A0A110C26000A0A120C26000A0A88
:10007000240C26000A0A200C26000A0A170C270066
:0E0080000000E702400A000000000000000837
:021FFE00EA0FE8
:00000001FF
